:1000000000308A008A2B0000A900030EAA00950B7D
:100010000D2819309500960A11140B112A0E830031
:10002000A90E290E090009000A108A100A11820778
:100030008734FF340A108A100A11820707340F34FC
:10004000003407340F34023407340F3404340734D7
:100050000F34083407340F34103407340F3420348D
:1000600007340F34053407340F3409340A108A106A
:100070000A11820709340234003430308400000849
:100080000319502801308D008C018C0B45288D0BF5
:1000900044280E308C008C0B4B280000800B42282B
:1000A00000348501860118306500FF306600831634
:1000B00081138312AD2B8C018D012B0803102C189A
:1000C0008C078C0C8D0CAC188C078C0C8D0C2C199F
:1000D0008C078C0C8D0CAC198C078C0C8D0C2C1A8D
:1000E0008C078C0C8D0CAC1A8C078C0C8D0C2C1B7B
:1000F0008C078C0C8D0CAC1B8C078C0C8D0C00347D
:1001000006089400FF3094061408F8399800980CFB
:10011000980C980C1F309805181E90280310980D05
:100120001808AB000330AC005B200D0898001408E1
:1001300007399E003C30A5001E08043C031CA5287E
:1001400005309F0001301E07A1001E08053C031D5D
:10015000AE2801309F00A1017830A5001E08053CA3
:100160000318BB281E08073C031CBB2802309F0055
:1001700005301E02A100AE2B8D018E018C018F0176
:100180003308031DC62832080319E0281030B400D4
:100190000310B00DB10D8C0D8F0D33080F02031D30
:1001A000D32832080C02031CDC2832088C02031C02
:1001B0008F0333088F0203148D0D8E0DB40BC828E6
:1001C0000000003419309500960197010130A0001D
:1001D0001115FF30A700003401302502A4000230C1
:1001E000B1005830B000B3012508B200BC200D08A2
:1001F000A800E22099010130A200810106308C00A4
:100200008C1D0A2907308101813084000008C03923
:100210000F3880006400813084000008C0390C046D
:1002200080008B168B17AF2B25081602031C232981
:1002300025089602970AA00A20081F0203182229FF
:100240000130A000111528081702031C2B29970163
:100250009908031D9903003410308C008F01B601FA
:10026000B30CB20C031C3A2934088F070318B60AE2
:100270003508B607B60C8F0C8E0C8D0C8C0B302904
:10028000003416082702031C70290330B100E8303F
:10029000B000B3011B08B200BC200E08B1000D086D
:1002A000B0000E08B3000D08B200B5012F08B4006D
:1002B0002C210E089D000D089C001D088F001C08B5
:1002C00003199D039C03B0000F08B100B008031D83
:1002D0006C29B108031970290130B0003D205D2957
:1002E000003416082702031CA3290330B100E830AC
:1002F000B000B3011B08B200BC200E08B1000D080D
:10030000B0000E08B3000D08B200B5012F08B4000C
:100310002C210E089D000D089C00051885141D0851
:100320008F001C0803199D039C03B0000F08B10047
:10033000B008031D9E29B1080319A2290130B0009D
:100340003D208F2985100034AE08031DAA290530F1
:10035000AF0041212E08803C0318BD292E08013C26
:100360000318BD290310AE0C031CB9291B08AF00EC
:1003700071210130AF004121AE292E08013C031844
:10038000D3290310AE0C031CCC290330AF0071211C
:100390000130AF004121D2290130AF00712101307D
:1003A000AF004121BD290230AF00412100340730A8
:1003B000AF004121920112088900831608148312AC
:1003C0000808FF3C0319EF29120889008316081456
:1003D00083120808AB00AE00A421920ADB29003486
:1003E00009309B0005140730AF0041212230AE00D8
:1003F000A421D7210510920105158519FD290511A4
:100400000608FF3A94001408013A03190E2A813AAB
:1004100003194A2A7F3A0319872A9F2A930113084E
:10042000023C031C492A13083620AB00120889003D
:100430002B0888000B088C008B130B088D0083168B
:10044000081555308900AA30890088148818262A92
:10045000081183120D088C1B8B0001301207AB00B2
:100460008900FF3088000B088C008B130B088D006F
:100470008316081555308900AA3089008814881819
:100480003F2A081183120D088C1B8B00920A930AD5
:100490000F2AD02A930113081420FF3C0319862A3F
:1004A00013081420AB00120889002B0888000B08E1
:1004B0008C008B130B088D008316081555308900AE
:1004C000AA30890088148818632A081183120D083D
:1004D0008C1B8B0001301207AB008900FF308800B5
:1004E0000B088C008B130B088D00831608155530F4
:1004F0008900AA308900881488187C2A0811831280
:100500000D088C1B8B00930A920A4B2AD02A1208E2
:100510008900140888000B088C008B130B088D00D1
:100520008316081555308900AA3089008814881868
:10053000972A081183120D088C1B8B00D02A1208F1
:100540008900140888000B088C008B130B088D00A1
:100550008316081555308900AA3089008814881838
:10056000AF2A081183120D088C1B8B000130120773
:10057000AB008900FF3088000B088C008B130B0840
:100580008D008316081555308900AA30890088141B
:100590008818C82A081183120D088C1B8B00920A38
:1005A0000514D7210510140FFC29BF2B8510051049
:1005B00091149118DD2A0511DE2A0515851DDE2A04
:1005C000E220180899002108A2009115BE2B990875
:1005D0000319282B19309B00142100301118013009
:1005E000013C031DFB2A023091069118F92A0511DE
:1005F000FA2A0515111099080319252B1908063C2C
:10060000031C252B180819020318252B210820028A
:10061000031D252B9608031D252B85100514073077
:10062000AF00412192011208023C031C242B210837
:10063000AB000330AC005B2012080D071A20AD00A0
:10064000AE00A421920A132B05109908031DEC2A71
:100650000511BF2BE2201421200822020319332B9D
:10066000A208031D882B003011190130013C031D25
:10067000882B851005140030111A0130003A031D33
:10068000582B19309B001608930089018316081413
:1006900083120808FF3C0319512BD7210330AF0008
:1006A0004121130824078D0016080D02A30011161E
:1006B00009309B002308A700230816020318762B95
:1006C0000730AF00412192011208023C031C752B38
:1006D0002108AB000330AC005B2012080D071A2084
:1006E000AD00AE00A421920A642B5C2B19309B0054
:1006F0002508A70089018316081483120808FF3C07
:10070000031DD72124081602031C822B051011118A
:100710002B2BC02B84011F30830511109110111158
:100720009111111292019301940195019601970183
:10073000980199019A019B019C019D019E019F01D5
:10074000A001A101A201A301A401A501A601A70185
:10075000A8010130B0003D2051288028EC288519DF
:10076000BF2B1608023C031CB92B8519B92B142189
:10077000B12B851DBD2B051AF029D62AE72A2A2B75
:02078000630014
:0A42000006000A0009001400FF0088
:02400E00F13F80
:00000001FF
